:020000040000FA
:0600000060283E300130D3
:08000800A000030EA100831209
:100010008B1C2E288B1031181328B11C2E2864300D
:100020000102031C2D281428152816281728182823
:1000300019281A281B283110B114A810031005190B
:100040000314AA0DA90DA80DB00B2E2831152A08EE
:10005000AF002908AE002808AD00B11081010B11D6
:0A006000210E8300A00E200E0900FF
:1000C000203084008001840A80300402031C6228EE
:1000D0001230B000FF2283160C3085058701831291
:1000E000850187010730990000309A00103083168F
:1000F0008E008312603083168F00831200308316C7
:1001000091009F008312C830831681008312313022
:100110009000003083168C00831210308B00BD1BC2
:100120009328851D84233D1BBE013D1BBF013D1F40
:100130006D2381018E018F010B118B100B108C012F
:100140008B17B2203119C820D122B30BAF2803106E
:1001500085190314BA0DF0303A0203190F22BD18A5
:10016000AC23A1286400311808000B1D08000B11F6
:10017000B11031141230B000051DC328321483169B
:10018000011383120800321083160117831208002E
:10019000321CCF282D090339AD00AE09AF09E43078
:1001A0002F02F0300319AF004C302F020C3003192E
:1001B000AF006C302F023C300319AF00EC302F023F
:1001C000FC300319AF00B3302F02F3300319AF0036
:1001D0001B302F020F300319AF003B302F023F308E
:1001E0000319AF00BB302F02FF300319AF003111EC
:1001F0000130B7008B132030370783169B001C1487
:100200001A088312A400A5002510103037078316A2
:100210009B001C141A088312A300003037078316B2
:100220009B001C141A088312A2008B1722082D02AF
:10023000031D092A23082E06FC39031D092A013053
:1002400009303702031D482900302E060339031DEB
:100250002D29BF1F3629BF13B11703302E060339CE
:10026000031D3629BF1B3629BF17B11744302F068F
:100270005439031D3F293F1F08003F13B1171030A9
:100280002F065439031D48293F1B08003F17B1179B
:10029000AF13AF12AF11AF1024082F02031DAA290C
:1002A00001303702031D59293E1859293E14B11750
:1002B000152302303702031D6229BE186229BE14BD
:1002C000B117172303303702031D6B293E196B2921
:1002D0003E15B117192304303702031D7429BE19C6
:1002E0007429BE15B1171B2305303702031D7D2964
:1002F0003E1A7D293E16B1171D2306303702031D15
:100300008629BE1A8629BE16B1171F230730370269
:10031000031D8F293E1B8F293E17B117212308305B
:100320003702031D9829BE1B9829BE17B117232336
:1003300009303702031DA1293F18A1293F14B11725
:1003400025230A303702031DAA29BF18AA29BF1482
:10035000B117292325082F02031D092A013037026E
:10036000031DB7293E1CB7293E10B1172D230230BB
:100370003702031DC029BE1CC029BE10B1172F2390
:1003800003303702031DC9293E1DC9293E11B1178B
:10039000312304303702031DD229BE1DD229BE11DC
:1003A000B117332305303702031DDB293E1EDB293D
:1003B0003E12B117352306303702031DE429BE1E55
:1003C000E429BE12B117372307303702031DED2988
:1003D0003E1FED293E13B117392308303702031DA4
:1003E000F629BE1FF629BE13B1173B230930370289
:1003F000031DFF293F1CFF293F10B1173D230A3081
:100400003702031D082ABF1C082ABF10B117412359
:10041000092AB70A0B30370203180800FA28B60178
:10042000B3019630B4000130B5000130B70085014A
:100430008701B113A122B220B30B592A03108519E9
:100440000314BA0DF0303A020319912AB40B592A59
:1004500001303702031945230230370203194923BB
:100460000330370203194D23043037020319512397
:100470000530370203195523063037020319592373
:100480000730370203195D2308303702031961234F
:1004900009303702031965230A303702031969232B
:1004A0003708B6080319B6000319572AB603963061
:1004B000B400311D1B2A3111321C632A2D09033966
:1004C000AD00AE09AF0951302F0655390319782A0E
:1004D00005302F0655390319782A15302F0655395E
:1004E0000319782A55302F0655390319782A1B2A03
:1004F000AF13AF12AF11AF108B1320303707BC0012
:100500002F08BB00DF2210303707BC002E08BB00CD
:10051000DF2200303707BC002D08BB00DF228B171D
:100520009B2285018701B70AB6010B303702031CF5
:100530001B2A6D2308000A303702031908008501C1
:1005400087016430B90033300F1E85000F1A850112
:10055000FF300F1A87000F1E8701B220311DA32A1A
:100560003111321CB82A2D090339AD00AE09AF098B
:1005700051302F0655390319A12A05302F06553958
:100580000319A12A15302F0655390319A12A553010
:100590002F0655390319A12AB90BA32A8501870112
:1005A0000800B11F0800B1131030BC003E08BB00AA
:1005B000DF223030BC003F08BB00DF2208003C08CF
:1005C0008B1383169B001C141A0883128B173B0293
:1005D000031908008B133B0883161C159A0083121D
:1005E0003C0883169B0055309D00AA309D009C144A
:1005F00064009C18F82A1C1183128B1708008316BC
:1006000000309B001C141A088312BD0083161030A2
:100610009B001C141A088312BE00831630309B0006
:100620001C141A088312BF0008000516080085165E
:100630000800051408008514080087140800071531
:1006400008000714080087160800BD1808000716E0
:100650000800BD180800871508000512080085125B
:100660000800051008008510080087100800071111
:1006700008000710080087120800BD1808000712BC
:100680000800BD180800871108000508103A850009
:1006900008000508203A850008000508013A850091
:1006A00008000508023A850008000708023A87009A
:1006B00008000708043A870008000708013A870085
:1006C00008000708203A870008000708103A87004A
:1006D00008000708083A870008003E180516BE18EB
:1006E00085163E190514BE1985143E1A8714BE1AC4
:1006F00007153E1B0714BE1B8716BD1808003F18C0
:100700000716BF1887150800B601B301B4013D1CD8
:100710008C2B3D10BD148F2BC030BD053D143D0802
:100720003F39B6006400942B952B962B972B982B72
:100730003330B41B8500B41F8501B30B922BB40B6F
:10074000922B0310B60CB608031D922B0030BC0090
:100750003D08BB00DF220800BF1FB72B3F1B07125D
:100760003F1B87153F1F07163F1F87110800071201
:0407700087110800E5
:084000000200000006000200AE
:02400E00CC33B1
:104200000100030003000300030003000300030098
:10421000030003000300FF00FF00FF00FF00FF009A
:10422000000000000000000000000000000000008E
:10423000000000000000FF00FF00FF00FF00FF0083
:104240000100510005001500550051000500150042
:10425000550051000500FF00FF00FF00FF00FF00B8
:104260000000FF00FF00FF00FF00FF00FF00FF0055
:10427000FF00FF00FF00FF00FF00FF00FF00FF0046
:10428000FF00FF00FF00FF00FF00FF00FF00FF0036
:10429000FF00FF00FF00FF00FF00FF00FF00FF0026
:1042A000FF00FF00FF00FF00FF00FF00FF00FF0016
:1042B000FF00FF00FF00FF00FF00FF00FF00FF0006
:1042C000FF00FF00FF00FF00FF00FF00FF00FF00F6
:1042D000FF00FF00FF00FF00FF00FF00FF00FF00E6
:1042E000FF00FF00FF00FF00FF00FF00FF00FF00D6
:1042F000FF00FF00FF00FF00FF00FF00FF00AA001B
:00000001FF
